:020000040000FA
:1000000099EF17F01200120014EF00F01200020036
:1000100064300000600000007F000000642F0000DA
:100020000004000000010000DACFE4FFE2CFDAFFB5
:10003000E9CFE4FFEACFE4FFF6CFE4FFF7CFE4FF38
:10004000F5CFE4FFF3CFE4FFF4CFE4FFFACFE4FF12
:1000500000EE18F0140EE80403E3EECFE4FFFBD744
:1000600000EE00F0180EE80403E3EECFE4FFFBD748
:10007000E652D9CFE6FFE1CFD9FFE6529EAA1BD0C8
:100080005AEC17F0DF6EAB50040B03E1AB50020BE0
:1000900002E0AB98AB88ACA2FED7010118C1E9FF22
:1000A00019C1EAFF182B000E1923000EE926040ED1
:1000B000EA22DFCFEFFFE552E552E7CFD9FFE55265
:1000C00000EE17F0180EE80403E3E5CFEDFFFBD7D1
:1000D00000EE2BF0140EE80403E3E5CFEDFFFBD7B1
:1000E000E5CFFAFFE5CFF4FFE5CFF3FFE5CFF5FF6E
:1000F000E5CFF7FFE5CFF6FFE5CFEAFFE5CFE9FF74
:10010000E5CFDAFF1100D59CD59AD596D584D58256
:10011000D580D66AD76AF29AD59EF1841200D9CFDB
:10012000E6FFE1CFD9FFFE0EDBCFE6FF79EC17F05B
:10013000E552FE0EDBCFE6FF79EC17F0E552FE0E3E
:10014000DBCFE6FF79EC17F0E552FE0EDBCFE6FFE2
:1001500079EC17F0E552E552E7CFD9FF1200180EFF
:10016000E66EA7EC17F0E55212000C0EE66EA7EC57
:1001700017F0E5521200180EE66EA7EC17F0E552E4
:100180001200D9CFE6FFE1CFD9FFFD0EDBCFE9FFAB
:10019000FE0EDBCFEAFFEFCF00F0000EE76E001897
:1001A000E8AE02D0003403D0E750D88000540FE20C
:1001B000FD0EDBCFE9FFDB2AFE0EDBCFEAFF01E31A
:1001C000DB2AEF50E66EA2EC16F0E552DED7E552E0
:1001D000E7CFD9FF12000B0EE66EA7EC17F0E55241
:1001E0001200D9CFE6FFE1CFD9FFE652FE0EDB5079
:1001F000DF6EDF380F0BDF1ADF50E840E8403F0BBF
:10020000DF1ADF407F0BDF1A010EDF14006E016A78
:1002100000C0F3FF01C0F4FF00D0E552E552E7CF84
:10022000D9FF1200D9CFE6FFE1CFD9FF060EE126B4
:10023000DE68DD68040EDB6A050EDB6A040EDBCFC8
:1002400000F0050EDBCF01F0FD0EDBCF02F0FE0E5D
:10025000DBCF03F00250005C0350015856E2040E5D
:10026000DBCFE9FF050EDBCFEAFF000EE926040E27
:10027000EA22EF50E76E000EDFCF00F0010EDBCF79
:1002800001F0E750001A00C0DEFF01C0DDFF080EDC
:10029000F36E020EF3CFDBFF030EDB6AD950020FC1
:1002A000E96EDACFEAFF000ED880EE54000EED546E
:1002B00026E2DF50010B10E0DECF00F0DDCF01F0D1
:1002C000D89001320032010E001AA00E011A00C0AF
:1002D000DEFF01C0DDFF0DD0D9CFE9FFDACFEAFFA5
:1002E000010E0F0B06E0EC52D890ED32EF32E8062B
:1002F000FAE1020EDB06030E01E2DB06CFD7040EA5
:10030000DB2A050E01E3DB2A99D7DECF2EF1DDCF04
:100310002FF1DECF00F0DDCF01F001C000F0016A67
:1003200000C030F1DECF00F0DDCF01F00050010160
:10033000316FFC0EDB042DE1FD0EDBCFE9FFFE0E7D
:10034000DBCFEAFF000EE926040EEA22EF50315D12
:100350001DE1010EE76EFD0EDBCFE9FFFE0EDBCFE8
:10036000EAFFE750E926000EEA22000EE926040E15
:10037000EA22EF50305D0AE1DECF00F0DDCF01F080
:1003800000C0F3FF01C0F4FF2BD02AD0F36AF46A57
:1003900027D0FD0EDBCFE9FFFE0EDBCFEAFF000E1C
:1003A000E926040EEA2231C1EFFF010EE76EFD0ED1
:1003B000DBCFE9FFFE0EDBCFEAFFE750E926000EB8
:1003C000EA22000EE926040EEA2230C1EFFFDECF5A
:1003D00000F0DDCF01F000C0F3FF01C0F4FF00D05A
:1003E000060EE15C02E2E16AE552E16EE552E7CF1A
:1003F000D9FF1200D9CFE6FFE1CFD9FF060EE126E3
:10040000FE0EDBCF00F4FD0EDBCF01F4FB0EDBCFE5
:1004100000F0FC0EDBCF01F001C000F0016A00C06B
:1004200002F4FF0EE76EFB0EDBCF00F0FC0EDBCF1D
:1004300001F0E7500016016A00C003F4F90EDBCFAB
:1004400000F0FA0EDBCF01F001C000F0016A00C03D
:1004500004F4FF0EE76EF90EDBCF00F0FA0EDBCFEF
:1004600001F0E7500016016A00C005F4FD0EDB50F4
:100470000F0801E07DD00401010E066F07C107F4EB
:10048000E66A080EE66EE66ACDDEE552E552E55212
:10049000F3CFDEFFF4CFDDFF0A0EF36E020EF3CFD3
:1004A000DBFF030EDB6A040EDB6A050EDB6A040E5B
:1004B000DBCF00F0050EDBCF01F0020EDBCF02F048
:1004C000030EDBCF03F00250005C035001581CE226
:1004D000E66A040EDBCFE9FF050EDBCFEAFF000E74
:1004E000E926040EEA22EF50E66E98EC09F0E55298
:1004F000E552200EE66EA2EC16F0E552040EDB2A61
:10050000050E01E3DB2AD3D7040EDB6A050EDB6A96
:10051000040EDBCF00F0050EDBCF01F0020EDBCFC7
:1005200002F0030EDBCF03F00250005C03500158D1
:1005300014E2040EDBCFE9FF050EDBCFEAFF000E6D
:10054000E926040EEA22EF50E66E6BD9E552040E5E
:10055000DB2A050E01E3DB2ADBD7020EDBCFE9FF46
:10056000030EDBCFEAFF000EE926040EEA22EF6A53
:10057000FD0EDB50030801E09FD06AD9080EF36E30
:10058000020EF3CFDBFF030EDB6AE66A060EE66EB1
:10059000E66A48DEE552E552E552F3CFDEFFF4CFDE
:1005A000DDFF00017A0ECA6F000ECB6F66C000F04F
:1005B00067C001F0026A00C0E6FF01C0E6FF02C0AA
:1005C000E6FFCAC0E6FFCBC0E6FF33EC17F0036ED0
:1005D000050EE15E0350CAC0E6FFCBC0E6FFD1DDE9
:1005E000E552E552090EE66EA2EC16F0E552040E55
:1005F000DB6A050EDB6A040EDBCF00F0050EDBCFF5
:1006000001F0020EDBCF02F0030EDBCF03F002504D
:10061000005C035001581CE2E66A040EDBCFE9FFE0
:10062000050EDBCFEAFF000EE926040EEA22EF50AA
:10063000E66E98EC09F0E552E552200EE66EA2EC6B
:1006400016F0E552040EDB2A050E01E3DB2AD3D7B0
:10065000040EDB6A050EDB6A040EDBCF00F0050E2C
:10066000DBCF01F0020EDBCF02F0030EDBCF03F095
:100670000250005C0350015814E2040EDBCFE9FF86
:10068000050EDBCFEAFF000EE926040EEA22EF504A
:10069000E66EC7D8E552040EDB2A050E01E3DB2A1D
:1006A000DBD7020EDBCFE9FF030EDBCFEAFF000E44
:1006B000E926040EEA22EF6A0101186B196B060E97
:1006C000E15C02E2E16AE552E16EE552E7CFD9FF73
:1006D0001200D9CFE6FFE1CFD9FF0A0EE126060EC0
:1006E000DB6A070EDB6A020EDB6A030EDB6ADE6A78
:1006F000DD6AFE0EDB500401005D3AE1030E015D90
:1007000037E1030E0225006E016A000E0122080E79
:1007100000C0DBFF090E01C0DBFF010EE66E080E14
:10072000DBCFE6FF090EDBCFE6FF7CDDE552E552CD
:10073000E552F3CFDEFFF4CFDDFFD9CFE9FFDACF0B
:10074000EAFF000ED880EE54000EED540DE20401D5
:100750000251E66ED950020FE96EDACFEAFFE55298
:10076000E750EE6EED6A04D0020EDB6A030EDB6A20
:10077000020EDBCF00F0030EDBCF01F000C0F3FF71
:1007800001C0F4FF0A0EE15C03E200D0E16AE55229
:10079000E16EE552E7CFD9FF1200810EE66EE66A00
:1007A0007E0EE66EBEEC16F0E552E552E552F28C96
:1007B000F28E1200D9CFE6FFE1CFD9FF020EE1267B
:1007C000DE6ADD6AFD0EDBCFE9FFFE0EDBCFEAFF5E
:1007D000EF5014E0FD0EDBCFE9FFFE0EDBCFEAFFAA
:1007E000EF50E66E1ED8E552DF2A010E01E3DB2A48
:1007F000FD0EDB2AFE0E01E3DB2AE4D7DECF00F09C
:10080000DDCF01F000C0F3FF01C0F4FF020EE15C98
:1008100003E200D0E16AE552E16EE552E7CFD9FF8D
:100820001200D9CFE6FFE1CFD9FFACA2FED7FE0E72
:10083000DBCFE6FFD6DCE552F350E8B0AC80E8A0B1
:10084000AC90FE0EDB50AD6EE552E7CFD9FF120043
:100850000A0EE66EA2EC16F0E5520D0EE66EA2EC64
:1008600016F0E5521200D9CFE6FFE1CFD9FF0A0E0C
:10087000E1260101CC0E006F000E016FFC0EDBCFF4
:1008800000F0010EE76E0018E8AE02D0003403D08D
:10089000E750D880005401E2D6D0FC0EDB5028E1AE
:1008A000FD0EDBCF00F0FE0EDBCF01F0060E00C028
:1008B000DBFF070E01C0DBFF080EDB6A090EDB6AF7
:1008C00000C1E6FF01C1E6FFD950060FE96EDACF9D
:1008D000EAFFEECFE6FFEECFE6FFEECFE6FFEFCF8B
:1008E000E6FFBBEC14F0006E060EE15E005010D087
:1008F00000C1E6FF01C1E6FFFD0EDBCFE6FFFE0E05
:10090000DBCFE6FF21EC14F0E552E552E552E5526B
:10091000010102AD84D0CC0EE66E000EE66E4CEC0A
:1009200017F0E552E552020EF3CFDBFF030EF4CFD2
:10093000DBFFDE6ADD6ADECF00F0DDCF01F0020E04
:10094000DBCF02F0030EDBCF03F00250005C03505C
:1009500001582EE2020EDBCF02F0030EDBCF03F0D4
:10096000DE50025CE96EDD500358EA6EE906000EC7
:10097000EA5ACC0EE926000EEA22EF50E66EFC0E93
:10098000DB50040F006E016A00BE0168DE50005C9F
:10099000E96EDD500158EA6ECC0EE926000EEA221F
:1009A000E552E750EF6EDF2A010E01E3DB2AC3D7E1
:1009B000DE6ADD6ADECF00F0DDCF01F0FC0EDB5039
:1009C000050F046E056A04BE0568020EDB50045C68
:1009D000026E030EDB500558036E0250005C03509C
:1009E00001581DE2010102A90BD0DECFE9FFDDCFE6
:1009F000EAFFCC0EE926000EEA22300EEF6E0AD096
:100A0000DECFE9FFDDCFEAFFCC0EE926000EEA22B9
:100A1000200EEF6EDF2A010E01E3DB2ACBD7FC0E9E
:100A2000DB50050FE96EEA6AE9BEEA68CC0EE926FA
:100A3000000EEA22EF6A00C1E6FF01C1E6FFC1EC49
:100A400000F0E552E5520A0EE15C02E2E16AE5528D
:100A5000E16EE552E7CFD9FF1200D9CFE6FFE1CF33
:100A6000D9FF0E0EE126F90EDBCFDEFFDBCFDDFF77
:100A7000F80EDBCF02F0000EE76E0218E8AE02D0EF
:100A8000023403D0E750D880025402E3070E12D09C
:100A9000F80EDBCF03F0160EE76E0318E8AE02D0B7
:100AA000033403D0E750D880035402E2170E02D07B
:100AB000F80EDB28006E016A00BE0168080E00C057
:100AC000DBFF090E01C0DBFF020EDB6A030EDB6AEF
:100AD000FB0EDBCF00F0FC0EDBCF01F0FD0EDBCF19
:100AE00002F0FE0EDBCF03F0226A236A246A256A35
:100AF00000C01DF001C01EF002C01FF003C020F0B6
:100B00003DEC13F0010A33E1F90EDBCFE9FFDB2AFC
:100B1000FA0EDBCFEAFF01E3DB2A2D0EEF6EFB0EB0
:100B2000DBCF00F0FC0EDBCF01F0FD0EDBCF02F0DF
:100B3000FE0EDBCF03F0226A236A800E246EBF0E06
:100B4000256E00C01DF001C01EF002C01FF003C0E2
:100B500020F061EC12F0FB0E1DC0DBFFFC0E1EC08E
:100B6000DBFFFD0E1FC0DBFFFE0E20C0DBFFFB0E18
:100B7000DBCF00F0FC0EDBCF01F0FD0EDBCF02F08F
:100B8000FE0EDBCF03F0226A236A246A256A00C0C6
:100B90001DF001C01EF002C01FF003C020F034ECB5
:100BA00013F0010A4AE1FB0EDBCF00F0FC0EDBCFB5
:100BB00001F0FD0EDBCF02F0FE0EDBCF03F0226A68
:100BC000236A800E246E3F0E256E00C01DF001C00A
:100BD0001EF002C01FF003C020F03DEC13F0010A2C
:100BE0002CE1006A016A200E026E410E036ED9509C
:100BF000FB0FE96EFF0EDA20EA6EEECF1DF0EECFAE
:100C00001EF0EECF1FF0EFCF20F000C022F001C0A9
:100C100023F002C024F003C025F061EC12F020C0E4
:100C2000EDFF1FC0EDFF1EC0EDFF1DC0EFFF020E68
:100C3000DB06030E01E2DB06B6D7FB0EDBCF00F0CE
:100C4000FC0EDBCF01F0FD0EDBCF02F0FE0EDBCFA2
:100C500003F0226A236A200E246E410E256E00C026
:100C60001DF001C01EF002C01FF003C020F03DECDB
:100C700013F0010A2EE0FB0EDBCF00F0FC0EDBCF01
:100C800001F0FD0EDBCF02F0FE0EDBCF03F0226A97
:100C9000236A200E246E410E256E00C01DF001C097
:100CA0001EF002C01FF003C020F00EEC12F0FB0E8D
:100CB0001DC0DBFFFC0E1EC0DBFFFD0E1FC0DBFFF7
:100CC000FE0E20C0DBFF020EDB2A030E01E3DB2A4F
:100CD000B4D7020EDBCF00F0030EDBCF01F0D9500A
:100CE000080FE96EDACFEAFF0050EE260150ED2240
:100CF000010EF36E040EF3CFDBFF050EDB6A040E6C
:100D0000DBCF1EF0050EDBCF1FF049EC11F00A0E11
:100D10001DC0DBFF0B0E1EC0DBFF0C0E1FC0DBFF78
:100D20000D0E20C0DBFF040EDBCF00F0050EDBCF85
:100D300001F0080EDBCF02F0090EDBCF03F001500B
:100D40000318E8AE02D0033404D00250005C035014
:100D500001582EE20A0EDBCF00F00B0EDBCF01F0C4
:100D60000C0EDBCF02F00D0EDBCF03F0226A236AFC
:100D7000200E246E410E256E00C01DF001C01EF035
:100D800002C01FF003C020F00EEC12F00A0E1DC0CE
:100D9000DBFF0B0E1EC0DBFF0C0E1FC0DBFF0D0EBA
:100DA00020C0DBFF040EDB2A050E01E3DB2ABBD7E4
:100DB0000A0EDBCF04F00B0EDBCF05F00C0EDBCF01
:100DC00006F00D0EDBCF07F0226A236A246A400E7C
:100DD000256E04C01DF005C01EF006C01FF007C040
:100DE00020F00EEC12F01DC000F01EC001F01FC07C
:100DF00002F020C003F0D950FB0FE96EFF0EDA209D
:100E0000EA6EEECF1DF0EECF1EF0EECF1FF0EFCF6B
:100E100020F000C022F001C023F002C024F003C083
:100E200025F078EC11F020C0EDFF1FC0EDFF1EC0D3
:100E3000EDFF1DC0EFFFFB0EDBCF00F0FC0EDBCFA4
:100E400001F0FD0EDBCF02F0FE0EDBCF03F0226AD5
:100E5000236A200E246E410E256E00C01DF001C0D5
:100E60001EF002C01FF003C020F03DEC13F0010A99
:100E700013E0FB0EDB6AFC0EDB6A800EF36EFD0EE8
:100E8000F3CFDBFF3F0EF36EFE0EF3CFDBFF020E60
:100E9000DB2A030E01E3DB2A020EDBCF00F0030E98
:100EA000DBCF01F00001800E01145FE0F90EDBCF13
:100EB000E9FFDB2AFA0EDBCFEAFF01E3DB2A300E83
:100EC000EF6EF90EDBCFE9FFDB2AFA0EDBCFEAFF8C
:100ED00001E3DB2A2E0EEF6E080EDBCF00F0090EC9
:100EE000DBCF01F0800E011414E0020EDBCF02F024
:100EF000030EDBCF03F0080EDB50025C006E090E20
:100F0000DB500358016E020E00C0DBFF030E01C070
:100F1000DBFF040EDB68050EDB68040EDBCF00F0A0
:100F2000050EDBCF01F0020EDBCF02F0030EDBCFAC
:100F300003F003500118E8AE02D0013404D0005091
:100F4000025C0150035811E2F90EDBCFE9FFDB2A06
:100F5000FA0EDBCFEAFF01E3DB2A300EEF6E040E60
:100F6000DB06050E01E2DB06D8D7040EDB6A050EB0
:100F7000DB6A040EDBCF00F0050EDBCF01F0080EBC
:100F8000DBCF02F0090EDBCF03F001500318E8AE0F
:100F900002D0033404D00250005C0350015801E336
:100FA000ACD0FB0EDBCF1DF0FC0EDBCF1EF0FD0E38
:100FB000DBCF1FF0FE0EDBCF20F0CEEC12F0060EE2
:100FC0001EC0DBFF070E1FC0DBFF300EE76E060EF4
:100FD000DBCF00F0070EDBCF01F0E7500026000E5C
:100FE0000122F90EDBCFE9FFDB2AFA0EDBCFEAFFA5
:100FF00001E3DB2A00C0EFFF040EDBCF00F0050E9B
:10100000DBCF01F0020EDB50001803E1030EDB50D2
:1010100001180BE1F90EDBCFE9FFDB2AFA0EDBCF7B
:10102000EAFF01E3DB2A2E0EEF6E060EDBCF1EF089
:10103000070EDBCF1FF049EC11F00A0E1DC0DBFFDD
:101040000B0E1EC0DBFF0C0E1FC0DBFF0D0E20C001
:10105000DBFF1DC000F01EC001F01FC002F020C069
:1010600003F0D950FB0FE96EFF0EDA20EA6EEECFE7
:101070001DF0EECF1EF0EECF1FF0EFCF20F000C03E
:1010800022F001C023F002C024F003C025F077EC69
:1010900011F020C0EDFF1FC0EDFF1EC0EDFF1DC011
:1010A000EFFF006A016A200E026E410E036ED950F6
:1010B000FB0FE96EFF0EDA20EA6EEECF1DF0EECFE9
:1010C0001EF0EECF1FF0EFCF20F000C022F001C0E5
:1010D00023F002C024F003C025F061EC12F020C020
:1010E000EDFF1FC0EDFF1EC0EDFF1DC0EFFF040EA2
:1010F000DB2A050E01E3DB2A3CD7F90EDBCFE9FF43
:10110000FA0EDBCFEAFFEF6A0E0EE15C02E2E16A63
:10111000E552E16EE552E7CFD9FF1200D9CFE6FFE5
:10112000E1CFD9FF060EE1260101029DFB0EDBCFC8
:101130001DF0FC0EDBCF1EF0FD0EDBCF1FF0FE0E10
:10114000DBCF20F0FDEC12F01CC0DEFF1DC0DEFF87
:101150001EC0DEFF1FC0DDFFDD52DD52FB0EDBCF08
:1011600004F0FC0EDBCF05F0FD0EDBCF06F0FE0E2B
:10117000DBCF07F0F90EDBCF1EF0FA0EDBCF1FF04E
:1011800049EC11F01DC008F01EC009F01FC00AF0A4
:1011900020C00BF008C022F009C023F00AC024F0E0
:1011A0000BC025F004C01DF005C01EF006C01FF0E6
:1011B00007C020F061EC12F01DC000F01EC001F06D
:1011C0001FC002F020C003F0F90EDBCF14F0FA0EBE
:1011D000DBCF15F0166A176A15AE02D016681768CD
:1011E00014C01CF015C01DF016C01EF017C01FF073
:1011F000DFCF21F0010EDBCF22F0020EDBCF23F098
:10120000030EDBCF24F0FBEC16F018C010F019C071
:1012100011F01AC012F01BC013F010C01CF011C066
:101220001DF012C01EF013C01FF05EEC11F01DC0C7
:101230000CF01EC00DF01FC00EF020C00FF00CC04F
:1012400022F00DC023F00EC024F00FC025F000C026
:101250001DF001C01EF002C01FF003C020F077ECAB
:1012600011F0CEEC12F0040E1EC0DBFF050E1FC005
:10127000DBFF7A0EE66E000EE66ED9CFE9FFDACF1D
:10128000EAFFEECFE6FFEECFE6FFEECFE6FFEFCFD1
:10129000E6FFBBEC14F0006E060EE15E00507A0E25
:1012A000E66E000EE66EC1EC00F0E552E5522E0E41
:1012B000E66EA2EC16F0E552F80EDBCFE6FFE66A2A
:1012C000040EDBCFE6FF050EDBCFE6FF33EC04F0C8
:1012D000E552E552E552E552060EE15C02E2E16AB2
:1012E000E552E16EE552E7CFD9FF1200D9CFE6FF14
:1012F000E1CFD9FFE652800EDF6EDF50000813E227
:10130000FE0EDB50DF1406E0310EE66EA2EC16F0A6
:10131000E55205D0300EE66EA2EC16F0E552DF4045
:101320007F0BDF6EEAD7E552E552E7CFD9FF120017
:10133000D9CFE6FFE1CFD9FF020EE126FE0EDB504A
:10134000F00BE8380F0B300FDF6EDF50390803E287
:10135000070EDF24DF6EFE0EDB500F0B300FE76E43
:10136000010EE7CFDBFFDB50390807E2010EDB504F
:10137000070FE76E010EE7CFDBFFDFCFE6FFA2EC42
:1013800016F0E552010EDBCFE6FFA2EC16F0E552B7
:10139000FD0EDB0405E1680EE66EA2EC16F0E552E8
:1013A000020EE15C02E2E16AE552E16EE552E7CF4E
:1013B000D9FF1200D9CFE6FFE1CFD9FFFB0EDBCF7B
:1013C0001DF0FC0EDBCF1EF0FD0EDBCF1FF0FE0E7E
:1013D000DBCF20F02034000E201809E6D880000E64
:1013E0001D54000E1E54000E1F54000E20540CE21B
:1013F000D950FB0FE96EFF0EDA20EA6EEE06000E02
:10140000EE5AEE5AEE5ADAD7E552E7CFD9FF12007C
:10141000D9CFE6FFE1CFD9FF020EE126DE6ADD6A11
:10142000DECF00F0DDCF01F0FE0EDB50000101AE9B
:1014300002D0D89003D0005C000E01580AE2200EC2
:10144000E66EA2EC16F0E552DF2A010E01E3DB2A7C
:10145000E7D7020EE15C02E2E16AE552E16EE55295
:10146000E7CFD9FF1200D9CFE6FFE1CFD9FFFE0EBB
:10147000DB50A96EA69EA69CA680F40EE66E010E19
:10148000E66EE66AE66A96DFE552E552E552E55217
:10149000A85000D0E552E7CFD9FF1200D9CFE6FF20
:1014A000E1CFD9FFFE0EDB50A96EFD0EDB50A86E1A
:1014B000A69EA684550EA76EAA0EA76EA682A1A808
:1014C000FED7A198A694E552E7CFD9FF1200D9CF55
:1014D000E6FFE1CFD9FFFB0EDBCFE9FFFC0EDBCF50
:1014E000EAFFEF501AE0FB0EDBCFE9FFDB2AFC0E30
:1014F000DBCFEAFF01E3DB2AEF50E66EFD0EDBCF28
:1015000000F0DB2AFE0EDBCF01F001E3DB2A005006
:10151000E66EC4DFE552E552DED7E552E7CFD9FFEC
:101520001200D9CFE6FFE1CFD9FF020EE126FD0E72
:10153000DBCFE6FF98DFE552DE6EDD6AD9CFE9FF4B
:10154000DACFEAFFEE50ED1001E11FD0DFCFE6FF6A
:10155000A2EC16F0E552FD0EDB2AFE0E01E3DB2ABB
:10156000FD0EDBCF00F0FE0EDBCF01F0013404E214
:101570000050FF08000E015401E207D0D9CFE9FF67
:10158000DACFEAFFEE50ED10D2E1980EE66E3A0E99
:10159000E66EE66AE66A0EDFE552E552E552E5528E
:1015A000020EE15C02E2E16AE552E16EE552E7CF4C
:1015B000D9FF1200BD6A8168DD0E936E938093920D
:1015C000938493869398938A938C938EC26A070E22
:1015D000C16E926E896A8268800E946E9490949225
:1015E000949494969498949A949C948E1200E2DF2A
:1015F0000101029F89988996CDEC03F083EC00F0FD
:101600009BEC16F0100EE66E270EE66EE66AE66AB2
:10161000D1DEE552E552E552E5520C0EE66EA2EC43
:1016200016F0E552F00EE66E490EE66E020EE66E1C
:10163000E66AC0DEE552E552E552E55228EC04F0D8
:1016400000017A0ECA6F000ECB6FCAC0E6FFCBC096
:10165000E6FFC1EC00F0E552E55228EC04F0000191
:101660007A0ECA6F000ECB6F60C000F061C001F04F
:10167000026A00C0E6FF01C0E6FF02C0E6FFCAC082
:10168000E6FFCBC0E6FF33EC17F0036E050EE15E1C
:101690000350CAC0E6FFCBC0E6FFC1EC00F0E55244
:1016A000E552898800017A0ECA6F000ECB6F62C0C6
:1016B00000F063C001F0026A00C0E6FF01C0E6FF6F
:1016C00002C0E6FFCAC0E6FFCBC0E6FF33EC17F06E
:1016D000036E050EE15E0350CAC0E6FFCBC0E6FF15
:1016E000C1EC00F0E552E552000EE66EE66A19DF45
:1016F000E552E552200EE66EE66A13DFE552E5524A
:10170000600EE66EE66A0DDFE552E552800EE66E8B
:10171000E66A07DFE552E55228EC04F00101386B78
:10172000396B8986D76AD66AD58E0101326B336BE5
:10173000186B196B010EE66EE66A000EE66EE66A3D
:10174000030EE66E010EE66EFAEC01F0006E060E78
:10175000E15E00500101186B196B880EE66E130EE6
:10176000E66EE66AE66A26DEE552E552E552E552A5
:10177000030EE66E010EE66E69EC03F0E552E552EB
:10178000F3CF14F1F4CF15F128EC04F000017A0E38
:10179000CA6F000ECB6F68C000F069C001F0026A2A
:1017A00000C0E6FF01C0E6FF02C0E6FFCAC0E6FFD8
:1017B000CBC0E6FF33EC17F0036E050EE15E03507D
:1017C000CAC0E6FFCBC0E6FFC1EC00F0E552E5522F
:1017D000090EE66EA2EC16F0E552040E0401022595
:1017E0000101166F176B000E17230E6B0F6B0E5156
:1017F000165D0F51175916E3E66A000E0E25E96EC5
:10180000040E0F21EA6EEF50E66E92DDE552E552CE
:10181000200EE66EA2EC16F0E55201010E2B000E32
:101820000F23E5D7090EE66EA2EC16F0E552000193
:101830007A0ECA6F000ECB6F6CC000F06DC001F065
:10184000026A00C0E6FF01C0E6FF02C0E6FFCAC0B0
:10185000E6FFCBC0E6FF33EC17F0036E050EE15E4A
:101860000350CAC0E6FFCBC0E6FFC1EC00F0E55272
:10187000E552090EE66EA2EC16F0E552E66A31C1B9
:10188000E6FF56DDE552E552200EE66EA2EC16F0BC
:10189000E552E66A30C1E6FF4BDDE552E55228EC41
:1018A00004F000017A0ECA6F000ECB6F6EC000F01C
:1018B0006FC001F0026A00C0E6FF01C0E6FF02C08F
:1018C000E6FFCAC0E6FFCBC0E6FF33EC17F0036EBD
:1018D000050EE15E0350CAC0E6FFCBC0E6FFC1ECD7
:1018E00000F0E552E552090EE66EA2EC16F0E55264
:1018F0000401035101011A6F1B6B04010451010122
:101900001C6F1D6B1AC101F0006A00501C25326F5C
:1019100001501D21336FE66A1AC1E6FF09DDE55269
:10192000E552200EE66EA2EC16F0E552E66A1CC106
:10193000E6FFFEDCE552E552090EE66EA2EC16F07B
:10194000E552E66AE66A32C1E6FF33C1E6FF33ECF0
:1019500004F0E552E552E552E552010E010132195B
:1019600001E1335139E0325101E1335101E035D029
:1019700028EC04F000017A0ECA6F000ECB6F76C01F
:1019800000F077C001F0026A00C0E6FF01C0E6FF88
:1019900002C0E6FFCAC0E6FFCBC0E6FF33EC17F09B
:1019A000036E050EE15E0350CAC0E6FFCBC0E6FF42
:1019B000C1EC00F0E552E55228EC04F08996400EA7
:1019C000E66E0D0EE66E030EE66EE66AF3DCE55299
:1019D000E552E552E55201D000D028EC04F00101B7
:1019E000000ED8803255000E335502E344EF11F05B
:1019F000186B196B010EE66EE66A500EE66EE66A2B
:101A0000030EE66E010EE66EFAEC01F0006E060EB5
:101A1000E15E0050880EE66E130EE66EE66AE66A38
:101A2000C9DCE552E552E552E5520101066B186B3F
:101A3000196B030EE66E010EE66E69EC03F0E552DB
:101A4000E552F3CF14F1F4CF15F128EC04F00001C6
:101A50007A0ECA6F000ECB6F68C000F069C001F04B
:101A6000026A00C0E6FF01C0E6FF02C0E6FFCAC08E
:101A7000E6FFCBC0E6FF33EC17F0036E050EE15E28
:101A80000350CAC0E6FFCBC0E6FFC1EC00F0E55250
:101A9000E552090EE66EA2EC16F0E552040E0401C2
:101AA00002250101166F176B000E17230E6B0F6BCB
:101AB0000E51165D0F51175916E3E66A000E0E25FA
:101AC000E96E040E0F21EA6EEF50E66E31DCE5524E
:101AD000E552200EE66EA2EC16F0E55201010E2B47
:101AE000000E0F23E5D7090EE66EA2EC16F0E552C4
:101AF00000017A0ECA6F000ECB6F6CC000F06DC093
:101B000001F0026A00C0E6FF01C0E6FF02C0E6FF86
:101B1000CAC0E6FFCBC0E6FF33EC17F0036E050E3C
:101B2000E15E0350CAC0E6FFCBC0E6FFC1EC00F0A7
:101B3000E552E552090EE66EA2EC16F0E552E66AB1
:101B400031C1E6FF98EC09F0E552E552200EE66E51
:101B5000A2EC16F0E552E66A30C1E6FF98EC09F017
:101B6000E552E55228EC04F000017A0ECA6F000E2F
:101B7000CB6F70C000F071C001F0026A00C0E6FFD8
:101B800001C0E6FF02C0E6FFCAC0E6FFCBC0E6FF29
:101B900033EC17F0036E050EE15E0350CAC0E6FF9A
:101BA000CBC0E6FFC1EC00F0E552E552090EE66E4F
:101BB000A2EC16F0E55204010351000EF350042587
:101BC0000101346F356B000E3523E66AE66A34C1D5
:101BD000E6FF35C1E6FF33EC04F0E552E552E5528D
:101BE000E552090EE66EA2EC16F0E552040E010174
:101BF000036A3625026E375103220751000802E3BB
:101C0000000E01D0010E046E056A04BE0568025084
:101C10000424006E03500520016E0050341902E1C7
:101C2000015035190BE14F0EE66EA2EC16F0E552AD
:101C30004B0EE66EA2EC16F0E55226D000017A0EAD
:101C4000CA6F000ECB6F78C000F079C001F0026A55
:101C500000C0E6FF01C0E6FF02C0E6FFCAC0E6FF23
:101C6000CBC0E6FF33EC17F0036E050EE15E0350C8
:101C7000CAC0E6FFCBC0E6FFC1EC00F0E552E5527A
:101C800034C136F135C137F134C136F135C137F1E0
:101C900028EC04F00101186B196B010EE66EE66A80
:101CA000E66EE66A030EE66E010EE66EFAEC01F0F1
:101CB000006E060EE15E0050880EE66E130EE66EB4
:101CC000E66AE66ADAEC09F0E552E552E552E552D9
:101CD0000101066B186B196B030EE66E010EE66EC2
:101CE00069EC03F0E552E552F3CF14F1F4CF15F1AE
:101CF00028EC04F000017A0ECA6F000ECB6F68C0AA
:101D000000F069C001F0026A00C0E6FF01C0E6FF12
:101D100002C0E6FFCAC0E6FFCBC0E6FF33EC17F017
:101D2000036E050EE15E0350CAC0E6FFCBC0E6FFBE
:101D3000C1EC00F0E552E552090EE66EA2EC16F099
:101D4000E552040E040102250101166F176B000E07
:101D500017230E6B0F6B0E51165D0F51175917E3BA
:101D6000E66A000E0E25E96E040E0F21EA6EEF50B2
:101D7000E66E98EC09F0E552E552200EE66EA2EC14
:101D800016F0E55201010E2B000E0F23E4D7090EC9
:101D9000E66EA2EC16F0E55200017A0ECA6F000E54
:101DA000CB6F6CC000F06DC001F0026A00C0E6FFAE
:101DB00001C0E6FF02C0E6FFCAC0E6FFCBC0E6FFF7
:101DC00033EC17F0036E050EE15E0350CAC0E6FF68
:101DD000CBC0E6FFC1EC00F0E552E552090EE66E1D
:101DE000A2EC16F0E552E66A31C1E6FF98EC09F084
:101DF000E552E552200EE66EA2EC16F0E552E66AD8
:101E000030C1E6FF98EC09F0E552E55228EC04F009
:101E100000017A0ECA6F000ECB6F72C000F073C063
:101E200001F0026A00C0E6FF01C0E6FF02C0E6FF63
:101E3000CAC0E6FFCBC0E6FF33EC17F0036E050E19
:101E4000E15E0350CAC0E6FFCBC0E6FFC1EC00F084
:101E5000E552E552090EE66EA2EC16F0E552E66A8E
:101E600004C4E6FF98EC09F0E552E552090EE66E6F
:101E7000A2EC16F0E55204C4E6FF76EC09F0E55258
:101E800028EC04F00101186B196B080EE66EE66A87
:101E9000030EE66EE66AE66E010EE66EFAEC01F0FF
:101EA000006E060EE15E0050880EE66E130EE66EC2
:101EB000E66AE66ADAEC09F0E552E552E552E552E7
:101EC0000101066B186B196B030EE66E010EE66ED0
:101ED00069EC03F0E552E552F3CF14F1F4CF15F1BC
:101EE00028EC04F000017A0ECA6F000ECB6F68C0B8
:101EF00000F069C001F0026A00C0E6FF01C0E6FF21
:101F000002C0E6FFCAC0E6FFCBC0E6FF33EC17F025
:101F1000036E050EE15E0350CAC0E6FFCBC0E6FFCC
:101F2000C1EC00F0E552E552090EE66EA2EC16F0A7
:101F3000E552040E040102250101166F176B000E15
:101F400017230E6B0F6B0E51165D0F51175917E3C8
:101F5000E66A000E0E25E96E040E0F21EA6EEF50C0
:101F6000E66E98EC09F0E552E552200EE66EA2EC22
:101F700016F0E55201010E2B000E0F23E4D7090ED7
:101F8000E66EA2EC16F0E55200017A0ECA6F000E62
:101F9000CB6F6CC000F06DC001F0026A00C0E6FFBC
:101FA00001C0E6FF02C0E6FFCAC0E6FFCBC0E6FF05
:101FB00033EC17F0036E050EE15E0350CAC0E6FF76
:101FC000CBC0E6FFC1EC00F0E552E552090EE66E2B
:101FD000A2EC16F0E552E66A31C1E6FF98EC09F092
:101FE000E552E552200EE66EA2EC16F0E552E66AE6
:101FF00030C1E6FF98EC09F0E552E55228EC04F018
:102000000101000ED8801455000E155501E3A3D030
:1020100000017A0ECA6F000ECB6F6AC000F06BC071
:1020200001F0026A00C0E6FF01C0E6FF02C0E6FF61
:10203000CAC0E6FFCBC0E6FF33EC17F0036E050E17
:10204000E15E0350CAC0E6FFCBC0E6FFC1EC00F082
:10205000E552E5520101106B116B89780E6B0F6B25
:1020600014510E5D15510F5976E2450EE66EA2EC45
:1020700016F0E552410EE66EA2EC16F0E552300E77
:1020800001011025E66EA2EC16F0E5523D0EE66E5B
:10209000A2EC16F0E552030E0101EA6A0E25E96E84
:1020A0000F51EA22000EE926040EEA22EF501A6FC1
:1020B0001B6B040EEA6A0E25E96E0F51EA22000E30
:1020C000E926040EEA22EF501C6F1D6B1AC103F0C3
:1020D000026A02501C25006E03501D21016E10C1C2
:1020E000E9FF11C1EAFF010ED890E936EA36E806A9
:1020F000FBE11E0EE926010EEA2200C0EEFF01C040
:10210000EDFFE66AE66A10C1E9FF11C1EAFF010EC0
:10211000D890E936EA36E806FBE11E0EE926010E04
:10212000EA22EECFE6FFEFCFE6FF33EC04F0E55214
:10213000E552E552E552090EE66EA2EC16F0E552C4
:102140000101102B000E1123020E0E250E6F000E42
:102150000F210F6F85D7386B396BF294D76AD66A27
:10216000D58E73EC16F00101076FD59EF2940751DE
:10217000000801E387D007512F0807E2400E075DF2
:1021800004E2300E075D076F0BD00751400807E2ED
:10219000470E075D04E2370E075D076F01D0076B3E
:1021A00028EC04F04B0EE66EA2EC16F0E552450E5C
:1021B000E66EA2EC16F0E552590EE66EA2EC16F0B1
:1021C000E5523D0EE66EA2EC16F0E552010EE66E0B
:1021D00007C1E6FF98EC09F0E552E55228EC04F05F
:1021E00000017A0ECA6F000ECB6F74C000F075C08C
:1021F00001F0026A00C0E6FF01C0E6FF02C0E6FF90
:10220000CAC0E6FFCBC0E6FF33EC17F0036E050E45
:10221000E15E0350CAC0E6FFCBC0E6FFC1EC00F0B0
:10222000E552E552090EE66EA2EC16F0E552040EF8
:10223000E66EE66A300EE66E010EE66E0F0EE66E94
:10224000010EE66EFAEC01F0006E060EE15E005043
:10225000880EE66E130EE66EE66AE66ADAEC09F0C0
:10226000E552E552E552E55228EC04F0500EE66ED8
:10227000C30EE66EE66AE66ADAEC09F0E552E5526C
:10228000E552E55228EC04F095EF0BF01200279E82
:1022900008D0279E1FAE05D01E6C1F1EE86A1F22A5
:1022A000278E1FC019F01EC018F02B6A2A6A8E0EE6
:1022B0001A6E1B6AB7EF13F0279E0CD0279E1FAE35
:1022C00009D01C6C1D1E1E1E1F1EE86A1D221E2228
:1022D0001F22278E1FC019F01EC018F01DC02BF042
:1022E0001CC02AF09E0E1A6E1B6AB7EF13F0257EF3
:1022F000276AF3EC13F00BEC14F027B69BEF13F006
:1023000027A20AD027AA03D027BE9BEF13F027A449
:10231000A7EF13F0A4EF13F027AA05D027ACA7EF7F
:1023200013F0A4EF13F027A00AD027A808D027BEE7
:1023300004D027A402D0B0EF13F0B4EF13F02A6A50
:102340001B6A2550205C296E10E31DC02BF01EC0B7
:1023500018F01FC019F020C028F022C01DF023C0C3
:102360001EF024C01FF0273A09D022C02BF023C052
:1023700018F024C019F025C028F0296C279E27BC2E
:10238000278E28C01AF027B0E3EF13F01A0E296049
:10239000E3EF13F01A6A206A27A408D01D6C1E1EF2
:1023A0001F1E201EE86A1E221F22202227AC08D0F2
:1023B0002B6C181E191E1A1EE86A182219221A22DE
:1023C0001C6A295207E020341F321E321D321C3293
:1023D000292EF9D71D502B261E5018221F501922C6
:1023E00020501A221CC02AF0279E1AAE0BD02A6C4D
:1023F0002B1E181E191E1A1EE86A2B2218221922DB
:102400001A22278E1AA006D0D880193218322B3201
:102410002A32282A28C01AF0B7EF13F0276AF3EC03
:1024200013F00BEC14F027B69BEF13F027A205D0A6
:1024300027BA9BEF13F0A2EF13F027BAAEEF13F019
:1024400027A005D027B89BEF13F0AEEF13F027B805
:10245000A2EF13F01B6A7F0E20241A6EE86A1B227B
:1024600025501A5EE86A1B5A1A0E286E206A2A6ADC
:102470002B6A186A196A22501D5E23501E5A245076
:102480001F5A000E205A09E722501D2623501E22F3
:1024900024501F22000E202201D02A8AD8901D36F7
:1024A0001E361F362036D8902A362B361836193667
:1024B000282EE1D71F501E101D10D8A42A8AB7EF6E
:1024C00013F0276AF3EC13F00BEC14F027B69BEF34
:1024D00013F027A205D027B89BEF13F0A2EF13F05B
:1024E00027AA05D027B09BEF13F0A2EF13F027B077
:1024F00002D027A802D0AEEF13F01B6A255020248B
:102500001A6EE86A1B227E0E1A5EE86A1B5A2A6A55
:102510002B6A186A196A24501F02F4CF19F0F3CFFE
:1025200018F023501F02F3502B26F4501822000EEF
:10253000192224501E02F3502B26F4501822000EAC
:10254000192222501F02F3502A26F4502B22000E8B
:102550001822192223501E02F3502A26F4502B224F
:10256000000E1822192224501D02F3502A26F4507E
:102570002B22000E1822192222501E02F4502A2665
:10258000000E2B221822192223501D02F4502A2655
:10259000000E2B2218221922B7EF13F0276AF3EC52
:1025A00013F027B6D8EF12F027A20ED027B405D02B
:1025B0007F0E1F6EFF0E1E6E1FD0800E1F6E1E6AD6
:1025C0001BD01F6A1E6A18D027B0FBD78F0E206061
:1025D000EDD77E0E2064F5D78E0E205C05E0D890F6
:1025E0001F321E32202AF8D727A406D01E6C1F1EC9
:1025F000E86A1F221FAEE5D71200276AF3EC13F03A
:1026000027B607EF13F027A20FD027B407D07F0E0D
:102610001F6EFF0E1E6E1D6E1C6E25D0800E1F6E6F
:1026200001D01F6A000EF6D727B0FBD71C6A9F0E99
:102630002060EBD77E0E2064F4D79E0E205C07E06E
:10264000D8901F321E321D321C32202AF6D727A402
:102650000AD01C6C1D1E1E1E1F1EE86A1D221E2293
:102660001F221FAEDED7120046EC13F027B6000C77
:1026700027B0000C27B4000C010C46EC13F027B671
:10268000000C27B0000C27A4000C010C276AF3EC07
:1026900013F00BEC14F027B6120027AE08D027A0D9
:1026A00004D027A802D027801200279012002550BE
:1026B000205C0BE124501F5C08E123501E5C05E107
:1026C00022501D5C02E127801200D8A002D0278E84
:1026D00010D0205025C020F0256E1F5024C01FF0C0
:1026E000246E1E5023C01EF0236E1D5022C01DF00C
:1026F000226E2550205C10E0FF0F09E0279027B4E0
:1027000003D027AE2784120027AE27941200252A73
:10271000D89024322332223222501D5E23501E5A7A
:1027200024501F5A1FBEEAD7D8901D361E361F36BA
:10273000202EF8D7C8D77F0E206EFF0E1F6E1E6E9C
:102740001D6E12007F0E27BEFF0E206E02D07F0E80
:10275000206E800E1F6E1E6A1D6AF3D727AE04D04E
:10276000800E206E1F6AF7D7206A1F6AF4D71950AF
:1027700018102B102A10F8E01BBEF0D719BE0CD091
:102780001A501B10EBE0D8902A362B361836193623
:102790001A06D8A01B06F2D71B50D4E11A28D2E0A3
:1027A0002AAE11D07F0E2A1402E12BA00CD02B2AC6
:1027B000E86A1822192207E3D880193218322B321E
:1027C0001A2A1A28BFE01A50C9E02BC01DF018C001
:1027D0001EF019341F6E1A30206E1F32209E27BE45
:1027E000208EA1EF13F01F36203602E32784277EC8
:1027F00006E12780206A1F6A1E6A1D6A12002028CF
:1028000003E0D8801F321200D8901F3202E12782E5
:102810001200278612002436253602E3278C277EF5
:1028200006E12788256A246A236A226A120025287D
:1028300003E0D88024321200D8902432EAE1278ABB
:102840001200D9CFE6FFDACFE6FFFA0EE3CFD9FFC9
:10285000FB0EE3CFDAFFFD0EE35209E72D0EDE6E2D
:10286000FC0EE31EE32AFD0ED8B4E306E31EE65297
:10287000E652E652FD0EE124E76EFF0EE220E46E22
:10288000E652F70EE3CFE6FFF70EE3CFE6FF91EC5B
:1028900014F0F90EE124E96EFF0EE220EA6E81ECFD
:1028A00014F00AE17EEC14F009E181EC14F008E187
:1028B0007EEC14F007E108D08CEC14F087EC14F0F7
:1028C0008CEC14F087EC14F08CEC14F0DE6AF90E4A
:1028D000E126FF0EE222FF0EE3CFDAFFE552FF0E04
:1028E000E3CFD9FFE552FC0EE124E96EFF0EE220B2
:1028F000EA6EEECFF3FFEFCFF4FF1200EF380F0BCD
:102900001200EF500F0B02E1EE52D8841200EF38A4
:102910000F0B300FDE6E1200EE500F0B300FDE6E1D
:102920001200FC0EE3CFE9FFFD0EE3CFEAFF100E2D
:10293000E66EEE6AEE6AEF6AD890FD0EE336FE0EA2
:10294000E336ED36ED36EF36FF0EE30609E0B2EC86
:1029500014F0EE52B2EC14F0EE52B2EC14F0EDD7EB
:10296000E56E1200030EEF24E8B6EF6E300EEF2492
:10297000E8BEEF6E000CD9CFE6FFDACFE6FFF80E27
:10298000E3CFD9FFF90EE3CFDAFFE652E652E65283
:10299000E652E652FB0EE124E76EFF0EE220E46E03
:1029A000E652F30EE3CFE6FFF30EE3CFE6FFF30EBE
:1029B000E3CFE6FFF30EE3CFE6FF40EC15F0F50EB4
:1029C000E124E96EFF0EE220EA6E2DEC15F019E12C
:1029D00030EC15F018E12DEC15F017E130EC15F0A6
:1029E00016E12DEC15F015E130EC15F014E12DECAD
:1029F00015F013E130EC15F012E12DEC15F011E1BA
:102A000012D036EC15F03BEC15F036EC15F03BEC43
:102A100015F036EC15F03BEC15F036EC15F03BEC10
:102A200015F036EC15F03BEC15F0DE6AF50EE126FC
:102A3000FF0EE222FF0EE3CFDAFFE552FF0EE3CFF7
:102A4000D9FFE552FA0EE124E96EFF0EE220EA6EAC
:102A5000EECFF3FFEFCFF4FF1200EF380F0B1200B1
:102A6000EF500F0B02E1EE52D8841200EF380F0B3B
:102A7000300FDE6E1200EE500F0B300FDE6E1200C4
:102A8000FA0EE3CFE9FFFB0EE3CFEAFF200EE66E7E
:102A9000EE6AEE6AEE6AEE6AEF6AD890FB0EE336F3
:102AA000FC0EE336FD0EE336FE0EE336ED36ED3674
:102AB000ED36ED36EF36FF0EE3060FE06FEC15F066
:102AC000EE526FEC15F0EE526FEC15F0EE526FEC2B
:102AD00015F0EE526FEC15F0E1D7E56E1200030E23
:102AE000EF24E8B6EF6E300EEF24E8BEEF6E000C78
:102AF000506F727420636F6D6D322048617264771D
:102B000061726520393630302C452C382C31203C10
:102B10002D3E2049544220206F7576657274200A3C
:102B20000D00506F727420636F6D6D3120536F66AE
:102B300074776172652031393230302C4E2C382C4C
:102B4000312020202D3E205662726179206F7576EB
:102B5000657274200A0D004331383A20313846320C
:102B600035385F4D6F646275735F4954425F43311E
:102B7000385F3132313133302E63200A0D00456E1B
:102B8000766F69205472616D6520284865786129E7
:102B90003A200052656365702E5472616D6520287D
:102BA00048657861293A20003820566F696573209E
:102BB000456E747265657320416E616C6F676971F3
:102BC00075657320313062697473203A0A0D0043D1
:102BD000524331363D2000535441545553203D203B
:102BE000004E62207472616D65732065786563754F
:102BF00074656573203D2000456E747265657320B1
:102C0000544F52204930202E2E204933203D2000A1
:102C1000536F727469657320544F52204F30202EC9
:102C20002E204F33203D200050524F424C454D4FF7
:102C3000202E2E2E2100457272657572205472610D
:102C40006D65202E2E2E21000E0EF66E000EF76EF4
:102C5000000EF86E00010900F550E46F0900F55010
:102C6000E56F03E1E46701D03DD00900F550DF6F67
:102C70000900F550E06F0900F550E16F0900090007
:102C8000F550E96E0900F550EA6E090009000900E7
:102C9000F550E26F0900F550E36F09000900F6CF27
:102CA000E6F0F7CFE7F0F8CFE8F0DFC0F6FFE0C0DE
:102CB000F7FFE1C0F8FF0001E25302E1E35307E050
:102CC0000900F550EE6EE207F8E2E307F9D7E6C037
:102CD000F6FFE7C0F7FFE8C0F8FF0001E407000EC9
:102CE000E55BBFD712000001080EEA6F0F010F016C
:102CF000F2B499EF16F00F0181BA77EF16F0EBEC12
:102D000000F00F0181BA77EF16F0BBEC00F00F0175
:102D100081AAD89081BAD8800001E933EA2F85EFE3
:102D200016F0BBEC00F0EBEC00F000000001E95104
:102D30001200000E12000F01939881880F01938AF0
:102D4000818A12000001FF0EE3CFE9F0090EEA6F5D
:102D5000D8900F01AEEF16F00001E9330F01D8A0B3
:102D60008198D8B08188AFEC00F00001EA2FACEF79
:102D700016F00F018188AFEC00F01200D9CFE6FF0A
:102D8000DACFE6FFE1CFD9FFE2CFDAFFAC6AAB6A78
:102D9000FD0EDBB0AC88DBA202D0AC8CAB8CDBB41C
:102DA000AC8EDBA602D0AB8801D0AB8ADBA802D008
:102DB000AC8401D0AC949E98DBAC02D09D8A01D04B
:102DC0009D9A9E9ADBAE02D09D8801D09D98FB0E05
:102DD000DB50AF6EAC8AAB8E949C948EAC50100BD3
:102DE00004E0AC50800B01E1948CE552E5CFDAFFB2
:102DF000E7CFD9FF12001C502102F3CF18F0F4CF17
:102E000019F02202F3501926000EF4201A6E1C50FD
:102E10002302F3501A26000EF4201B6E1C502402CD
:102E2000F3501B261D502102F3501926F4501A228C
:102E3000000E1B221D502202F3501A26F4501B22B2
:102E40001D502302F3501B261E502102F3501A2658
:102E5000F4501B221E502202F3501B261F50210249
:102E6000F3501B261200FB0EE3CFF6FFFC0EE3CF60
:102E7000F7FFFD0EE3CFF8FFFE0EE3CFE9FFFF0EF5
:102E8000E3CFEAFFE9CFF3FFEACFF4FF0900F5CF84
:102E9000EFFFEE66FBD71200FE0EE3CFE9FFFF0E59
:102EA000E3CFEAFFF36AF46AEE5203E0F34AF42A4E
:102EB000FBD71200D9CFE6FFDACFE6FFE1CFD9FF8B
:102EC000E2CFDAFFE652F20E0001EB17ABAC03D013
:102ED000EB91ABB0EB81ABB4EB85ABB2EB87AE5013
:102EE000DF6EDF50E552E552E5CFDAFFE7CFD9FFDD
:102EF0001200FF0EE3502C6E480E01D04C0EE76E10
:102F0000E72EFED7E76AE72EFED72C2EF7D7000074
:102F10001200000EF36E00EE00F0060E01D8120053
:102F2000EA6002D0EE6AFCD7F350E9601200EE6A64
:102F3000FCD715EE00F025EE00F0F86A279C24EC93
:102F400016F003EC00F0F7EC0AF0FBD71200FF0ECE
:102F5000E350E84E1200000000D000D000D0E82E70
:102F6000FAD712000000000000000000000000007E
:102F70000000000000000000000000000000000051
:102F80000000000000000000000000000000000041
:102F90000000000000000000000000000000000031
:102FA0000000000000000000000000000000000021
:102FB0000000000000000000000000000000000011
:102FC0000000000000000000000000000000000001
:102FD00000000000000000000000000000000000F1
:102FE00000000000000000000000000000000000E1
:102FF00000000000000000000000000000000000D1
:1030000000000000000000000000000000000000C0
:1030100000000000000000000000000000000000B0
:1030200000000000000000000000000000000000A0
:103030000000000000000000000000000000000090
:103040000000000000000000000000000000000080
:103050000000000000000000000000000000000070
:1030600000000000F02A222B572B7E2B932BA82B3D
:10307000CF2BD72BE12BF82B102C282C362C3138CA
:10308000463235385F4D6F646275735F4954425FF5
:103090004331385F3132313230312E6320202020ED
:1030A0002020202020202020000000000000000020
:1030B0000000000000000000000000000000000010
:1030C00000000000000000000000000000007A0086
:1030D00031323334353637383930313233343536AE
:1030E000000000FFFFFFFFFFFFFFFFFFFFFFFFFFED
:1030F000FFFFFFFFFFFFFFFFFFFFFFFFFFFFFFFFE0
:10310000FFFFFFFFFFFFFFFFFFFFFFFFFFFFFFFFCF
:10311000FFFFFFFFFFFFFFFFFFFFFFFFFFFFFFFFBF
:10312000FFFFFFFFFFFFFFFFFFFFFFFFFFFFFFFFAF
:0200000400F00A
:1000000050726F6A65743A3138463235785F4D6F99
:10001000646275732E6D63702020202020200D00F7
:10002000506F727420436F6D3220393630302C455A
:1000300076656E205061726974792C382C310D0010
:1000400041766563205541525420484152445741FE
:100050005245203C2D3E20495442202020200D00B6
:100060005642726179203C2D3E5541525420536FC7
:1000700066742031393230302C4E2C382C310D0042
:10008000313846323538202B205069636B69742033
:10009000322E3631202020202020202020200D004C
:1000A0007061756C666A756A6F40667265652E660A
:1000B00072202020202020202020202020200D0021
:1000C0004D504C4142204944452056382E38343357
:1000D00020204331382076332E34312020200D006B
:1000E0002020202020202020202020202020202010
:1000F000202020202020202020200D0A00000000A9
:020000040030CA
:0E0000000022040E000081000FC00FE00F4030
:020000040020DA
:08000000FFFFFFFFFFFFFFFF00
:00000001FF
